:100000000A128A11452BFF1B0D2883137F188317B3
:100010000008840A0319FF0A080000308A00040857
:10002000840A82070034CF340034DB340034E634F1
:100030000034F6340034053401341F3401342F34D5
:10004000013448340134783401349F340134C834E5
:100050000134FF3401344F340234CF3402343F349E
:100060000334FF340334493444343A34503449348B
:10007000433431343634463438343834363420342A
:100080005534413452345434203474346534733428
:100090007434203400340A340A345034493443343C
:1000A00031343634463438343834363420345534E8
:1000B00041345234543420347434653473347434D9
:1000C0002034003455346E346B346E346F347734EE
:1000D0006E34203463346F346D346D3461346E3477
:1000E00064340A34003420346D347934203461347B
:1000F000643472346534733431343D3400346D34D7
:100100007934203461346434723465347334303477
:040110003D34003446
:10061200563431342E3436343434733470346934CD
:10062200003477080A128A1120240A128A117608E5
:100632000A128A1120240A128A110800F000700896
:10064200831203139300262B640083160313141CD6
:100652002B2B2C2B252B2D2B831203131308312B21
:1006620008007E088A007F0882000A128A1132235B
:100672000A128A118000840A04087D0603190034D4
:10068200FF0A0319FE0A362BFC0183133430FD00E6
:100692000330FE000930FF002B3084000A128A1159
:1006A20036230A128A1183010A128A11F52DF100EA
:1006B2007B30710203185E2B5F2B6A2B6130710253
:1006C200031C642B652B6A2BDF30F0007008F105E8
:1006D2006A2B71086C2B0800831203139412831681
:1006E200031306138713831203131416141094149E
:1006F2001411941183160313941314178312031302
:10070200941608000C3083160313990018158316EB
:10071200031787110710831603131812831203138A
:10072200981718169812831603130C128C121813AA
:1007320083120313181383160313981298160800D2
:10074200F100BE2B981CA62BA72BAF2B83160313ED
:10075200981298168312031318121816181DB22B2A
:10076200B32BBC2B1A08F0007008FC00831603138D
:1007720098129816BC2B6400BE2B831203130C1E16
:10078200C32BC42BA32BC52B710899000800E62BA1
:10079200640083120313981CCF2BD02BD82B831603
:1007A2000313981298168312031318121816181DA1
:1007B200DB2BDC2BE62B1A08F0007008FC008316FA
:1007C200031398129816E62BE62B831203138C1E42
:1007D200EB2BEC2BC92BED2B1A08EF2B08000B2C63
:1007E20075080A128A11A1230A128A1175080A3A97
:1007F200031DFC2BFD2B042C0D300A128A11A123A0
:100802000A128A11042C0130F2070318F30A00308D
:10081200F3070B2C730883120313FF007208840082
:100822000A128A1103200A128A11F4007408F500D0
:10083200F508031D1D2C1E2CF12B1F2C0800F500A2
:100842007508F2007208F4007508F2000430031013
:10085200F20CFF3E031D282C7208F3007308F5000A
:100862000A3075020318362C372C3C2C3030F2003B
:100872007208F507412C3730F2007208F507412C57
:1008820075080A128A11A1230A128A117408F20049
:100892007208F50075080F39F2007208F5000A3087
:1008A20075020318552C562C5B2C3030F20072085E
:1008B200F507602C3730F2007208F507602C7508D6
:1008C2000A128A11A1230A128A110800FF30F500C8
:1008D2000030F600F701F8010030780210300319F9
:1008E2007702031C752C762C782CAA2CAA2C77085C
:1008F200F2007207013E84000A128A110D200A12C8
:100902008A11F3000A128A110D200A128A11F400C8
:1009120071087402031D8F2C70087302031C922C41
:10092200932C9A2C7808F601F6077708F501F5075B
:10093200AA2C0130F7070318F80A0030F807003034
:100942007802103003197702031CA82CA92C782CEA
:10095200AA2C7608F101F1077508F001F007B12C15
:100962000800F4000F30F2007208F405C130F20002
:100972007208831203139F057408F20001300310FA
:10098200F20DFF3E031DC02C0310720DF30073081D
:100992009F041F139F17831603139F1783120313BA
:1009A2001F14831603130C13831203130C138316E1
:1009B20003139E01831203139E010630F200F20B11
:1009C200E02C6400831203139F14E72C9F18EA2C77
:1009D200EB2CE72CEC2C1E08F200F3017208F3005A
:1009E200F201831603131E087207F0000030031889
:1009F20001307307F100FD2C0800F4010A128A117C
:100A0200C8230A128A110A128A1158230A128A1159
:100A1200F2007208F50030307502031C112D122D00
:100A22001E2D3A3075020318172D182D1E2D75082C
:100A3200D03EF2007208F400302D41307502031CE2
:100A4200232D242D302D473075020318292D2A2DF0
:100A5200302D7508C93EF2007208F400302D74087A
:100A6200F20003300310F20DFF3E031D332D03107D
:100A7200720DF3007308F4000A128A11C8230A12D5
:100A82008A110A128A1158230A128A11F200720874
:100A9200F50030307502031C4F2D502D5C2D3A307D
:100AA20075020318552D562D5C2D7508D03EF200A7
:100AB2007208F5006E2D41307502031C612D622D06
:100AC2006B2D473075020318672D682D6B2D37305B
:100AD200F5026E2DF5016E2D6E2D0F30F2007208AB
:100AE200F5057508F2007208F4047408782D080000
:100AF200F000F008031D7E2D7F2D832D8316031336
:100B02000514F02D7008013A031D882D892D8D2DB5
:100B1200831603138514F02D7008023A031D922DDB
:100B2200932D972D831603130515F02D7008033AA4
:100B3200031D9C2D9D2DA12D831603138515F02DCC
:100B42007008043A031DA62DA72DAB2D831603139F
:100B52008516F02D7008083A031DB02DB12DB52D64
:100B6200831603130615F02D7008093A031DBA2DDA
:100B7200BB2DBF2D831603138615F02D70080A3A7C
:100B8200031DC42DC52DC92D831603138614F02D04
:100B920070080B3A031DCE2DCF2DD32D83160313D0
:100BA2000616F02D70080C3A031DD82DD92DDD2D17
:100BB200831603130614F02D70080D3A031DE22D5F
:100BC200E32DF02D831603138616F02DF02DF02D54
:100BD200F02DF02DF02DF02DF02DF02DF02D8316AF
:100BE20003131F129F12080083120313A901AA0103
:100BF200831603130F178F160F160513871287110B
:100C020085130A128A1183230A128A110330FB0008
:100C12008A30FA005630F900F90B0D2EFA0B0D2E20
:100C2200FB0B0D2E142E0A128A116D230A128A1141
:100C32000330FB008A30FA005630F900F90B1F2E00
:100C4200FA0B1F2EFB0B1F2E262E00300A128A11C2
:100C52001F230A128A1183120313A901AA01003069
:100C62002A020E3003192902031C382E392E3B2E7C
:100C7200532E532E00300A128A1179250A128A1134
:100C8200013083120313A9070318AA0A0030AA0726
:100C920000302A020E3003192902031C512E522E53
:100CA2003B2E532E3930F2008030F3000A128A11A3
:100CB200F0230A128A112B30F2000030F3000A12DC
:100CC2008A11F0230A128A1100300A128A11B22400
:100CD2000A128A11710883120313A101A107700875
:100CE200A001A00701300A128A11B2240A128A1145
:100CF200710883120313A301A3077008A201A207BC
:100D02002108F101F1072008F001F0070A128A1107
:100D120067240A128A11710883120313A801A80713
:100D22007008A701A7072308F101F1072208F001C3
:100D3200F0070A128A1167240A128A1171088312B3
:100D42000313A601A6077008A501A5076D30F200DE
:100D52008030F3000A128A11F0230A128A118312D8
:100D620003132808F701F7072708F601F6070A1206
:100D72008A1112230A128A116130F2008030F300C4
:100D82000A128A11F0230A128A1183120313260807
:100D9200F701F7072508F601F6070A128A1112234E
:100DA2000A128A115F30F2008030F3000A128A11AF
:100DB200F0230A128A11DD2E0A128A11C8230A129E
:100DC2008A110A128A1158230A128A11F900790823
:100DD20083120313A400E02F8513F930F900640095
:100DE200F90BF02EF42E6400DD2E8517F930F90090
:100DF2006400F90BF92EFD2E6400DD2E0A128A1111
:100E0200FE240A128A110A128A111F230A128A1157
:100E1200F930F9006400F90B0B2F0F2F6400DD2E5F
:100E2200023083120313A9000030AA0000302A0204
:100E32000E3003192902031C1F2F202F222F592F96
:100E4200592F29080A128A1120240A128A113A30CB
:100E52000A128A11A1230A128A1183120313290882
:100E62000A128A11B2240A128A117108F701F707CD
:100E72007008F601F6070A128A1112230A128A1161
:100E82003B300A128A11A1230A128A1101308312FD
:100E92000313A9070318AA0A0030AA0700302A027E
:100EA2000E3003192902031C572F582F222F592FB6
:100EB2005F30F2008030F3000A128A11F0230A1226
:100EC2008A11DD2E83120313A901AA01792F68303A
:100ED200FA00E430F900F90B6C2FFA0B6C2F640066
:100EE200013083120313A9070318AA0A0030AA07C4
:100EF2002A082802031D7F2F290827020318822FA0
:100F0200832F682F842F2130F2008030F3000A12E1
:100F12008A11F0230A128A112B30F2000030F300FA
:100F22000A128A11F0230A128A116F30F2008030FD
:100F3200F3000A128A11F0230A128A118312031390
:100F42002808F701F7072708F601F6070A128A119F
:100F520012230A128A116430F2008030F3000A125E
:100F62008A11F0230A128A11831203132608F70149
:100F7200F7072508F601F6070A128A1112230A1248
:100F82008A115F30F2008030F3000A128A11F023D6
:100F92000A128A11DD2E20300A128A11A1230A12A6
:100FA2008A11DD2EDD2EDD2E5030F2008030F3006E
:100FB2000A128A11F0230A128A11DD2EDD2E831203
:100FC200031324080A3A0319DD2E073A0319DD2E0A
:100FD2002D3A0319CC2F643A0319ED2E013A031965
:100FE200F62E0C3A0319632F1B3A0319112F013AFB
:0E0FF2000319FF2ED52FDD2E0A128A110028BA
:084000000E000D000100070095
:04400E00ECEBFFFEDA
:00000001FF
